:020000020000FC
:0200000002C03C
:1000040018950CEF0ABB03E00BBB07E007BB0FE03E
:1000140008BB00E808B90FED0DBF02E002BB00E128
:100024000BBFBB2770E08AED9AE9A3E0C89904C02E
:10003400DA9A00C0C899B360DA98B0FF96D142D07A
:1000440024D06AD005D04CD02CD058D00DD0F7CFC6
:1000540023E03FE36FD012E315D130E06BD012E31D
:1000640011D12A95B1F7089523E030E063D012E06E
:1000740009D133953F33D1F75DD012E003D13A95DE
:100084000000D1F72A9591F708952AE030E077D05F
:100094001FE0F8D03FE373D01FE0F4D02A95B1F706
:1000A400089525E030E06BD012E0ECD033953F3377
:1000B400D1F765D012E0E6D03A950000D1F72A9541
:1000C40091F7089525E0C0E630E034D03FE3398766
:1000D400399314E1D7D0C936B9F72A95A1F7089511
:1000E40025E0C9E630E026D03FE33A93398714E1AE
:1000F400C9D0C036B9F72A95A1F7089525E030E0B4
:1001040019D0C0E664D03FE3399314E1BBD0C237C1
:10011400C9F72A95B1F7089525E030E00BD0C2E77E
:1001240056D03FE33A9314E1ADD0C036C9F72A95CF
:10013400B1F708953093600030936100309362000A
:10014400309363003093640030936500309366000D
:1001540030936700309368003093690030936A00ED
:1001640030936B0030936C0030936D0030936E00CD
:1001740030936F0030937000309371000895032F13
:1001840000950F7330936000009361003093620018
:10019400009363003093640000936500309366001D
:1001A40000936700309368000093690030936A00FD
:1001B40000936B0030936C0000936D0030936E00DD
:1001C40000936F0030937000009371000895309194
:1001D400600036953093600030916100369530931D
:1001E4006100309162003695309362003091630073
:1001F40036953093630030916400369530936400F3
:1002040030916500369530936500309166003695DF
:1002140030936600309167003695309367003091D3
:1002240068003695309368003091690036953093B4
:10023400690030916A00369530936A0030916B0002
:10024400369530936B0030916C00369530936C008A
:1002540030916D00369530936D0030916E00369577
:1002640030936E0030916F00369530936F0030916B
:10027400700036953093700030917100369530934C
:100284007100089502D01A95E9F75EE340EC0091FD
:1002940060005017479500916100501747950091F1
:1002A40062005017479500916300501747950091DD
:1002B40064005017479500916500501747954BBB54
:1002C400C09840EC00916600501747950091670074
:1002D40050174795009168005017479500916900A1
:1002E4005017479500916A005017479500916B008D
:1002F40050174795C09A4BBBC19840EC00916C00D5
:100304005017479500916D005017479500916E0066
:100314005017479500916F00501747950091700052
:10032400501747950091710050174795C19A4BBBE0
:10033400C298C99907C067FF63956F3731F4B0FF5E
:1003440014D003C0662700C000008894B1FF715028
:1003540080409040A04009F408D006D000C00000BE
:10036400C29A515008F092CF0895C29A03E00BBB91
:10037400C99BFECFD898D09A00E10ABF789400E3D5
:1003840005BF889500E105BF662700E00A95F1F7EF
:100394000DE40A95F1F7C999F2CF63956233A8F396
:1003A4006FEFD098D89AF89470E08AED9AE9A3E0B8
:0803B400BD7FC89BB2600895F3
:00000001FF
